:03000000021CF4EB
:101CF40078FFE4F6D8FD9000007F007E04E4F0A3B2
:101D0400DFFCDEFA750804750900758120021D4F99
:0B237F00480136A0D0E8F4FAFDFEFF94
:1020530090FFFE121959EEF0A3EFF090FFFF121953
:012063005923
:10206400C0A8C2AF850883850982A3E0FEA3E0FF70
:102074002406F582E43EF583E0FCA3E0FDEF2404AE
:10208400F582E43EF583E0FEA3E0B50508EEB50471
:10209400047F0180027F00850883850982EFF0D0E8
:0920A400A8850883850982E0FF8C
:0620AD0090000302195926
:1013380090FFFF121959EDF090FFFE121959EEF0C7
:09134800A3EFF090FFFE12195909
:10135100C0A8C2AF850883850982A3A3E0FEA3E0EC
:10136100FF2406F582E43EF583E0FCA3E0FD850859
:1013710083850982ECF0A3EDF08F828E83A3A3E035
:10138100FEA3E0FF850883850982A3A3E0FAA3E019
:10139100F5828A83E0FAA3E02FFFEA3ECF2401CF52
:1013A1003400FEED2401FDE43CFCEDB5072AECB56B
:1013B1000626850883850982A3A3E0FEA3E0FFF545
:1013C100828E83E0FCA3E0FDEF2406F582E43EF586
:1013D10083ECF0A3EDF0801B850883850982A3A32C
:1013E100E0FEA3E02406F582E43EF583E475F00116
:1013F100121910850883850982A3A3E0FEA3E0FFEB
:10140100122053EF602A850883850982E0FEA3E05C
:10141100FF850883850982A3A3E0FCA3E02406F5E8
:1014210082E43CF583EEF0A3EFF0D0A87F00801CAE
:1014310090000412197DE0FF850883850982E0FC94
:0C144100A3E0F5828C83EFF0D0A87F01BF
:06144D0090000502195990
:10163F0090FFFE121959ECF0A3EDF090FFFE121976
:10164F0059EEF0A3EFF0C0A8C2AF850883850982D9
:10165F00E0FEA3E0FF122053EF6007D0A87F000247
:10166F001725850883850982E0FEA3E0FF2404F592
:10167F0082E43EF583E0FCA3E0F5828C83E0FD85F8
:10168F000883850982A3A3E0FAA3E0F5828A83ED9C
:10169F00F08F828E83A3A3E0FEA3E0FF85088385EE
:1016AF000982E0FCA3E0FDF5828C83E0FAA3E02F32
:1016BF00FFEA3ECF2401CF3400FEED2404F582E48F
:1016CF003CF583E0FCA3E02401FDE43CFCEDB50711
:1016DF0028ECB50624850883850982E0FEA3E0FF88
:1016EF00F5828E83E0FCA3E0FDEF2404F582E43E57
:1016FF00F583ECF0A3EDF08019850883850982E06E
:10170F00FEA3E02404F582E43EF583E475F00112B4
:0C171F001910D0A87F0190000402195995
:10211100900003E4F0A37424F07E007F119000018D
:10212100EEF0A3EFF0900007EEF0A3EFF0900005C2
:10213100EEF0A3EFF090000BE4F0A374FFF07E004B
:102141007F36900009EEF0A3EFF090000FEEF0A3C0
:10215100EFF090000DEEF0A3EFF090013E7401F06E
:03216100A3F022C6
:1023C40090013EE0B40108D2B30000E4F0D29922B7
:03002300021F6A4F
:101F6A00C0E0C0F0C083C082C0D075D000C000C03D
:101F7A0001C002C003C004C005C006C00730992FC3
:101F8A007E007F09122053EF700E90000DE0FEA331
:101F9A00E0F5828E83E0F599C2997C017D407E004E
:101FAA007F0912163FEF700790013E04F0C2B3306A
:101FBA00980EC298AD997E007F011213381223E45D
:101FCA00D007D006D005D004D003D002D001D0006B
:0B1FDA00D0D0D082D083D0F0D0E03215
:1023980075985075892075878090013DE0F58D7599
:0723A8008840D2ACD2AF2245
:10000E00759A50758E1890013DE0F59C538EFB75D8
:05001E00AF01D2AF228A
:0B240100122111122398121A4A80FBCE
:100D630000C1814001C0804101C0804100C1814078
:100D730001C0804100C1814000C1814001C0804168
:100D830001C0804100C1814000C1814001C0804158
:100D930000C1814001C0804101C0804100C1814048
:100DA30001C0804100C1814000C1814001C0804138
:100DB30000C1814001C0804101C0804100C1814028
:100DC30000C1814001C0804101C0804100C1814018
:100DD30001C0804100C1814000C1814001C0804108
:100DE30001C0804100C1814000C1814001C08041F8
:100DF30000C1814001C0804101C0804100C18140E8
:100E030000C1814001C0804101C0804100C18140D7
:100E130001C0804100C1814000C1814001C08041C7
:100E230000C1814001C0804101C0804100C18140B7
:100E330001C0804100C1814000C1814001C08041A7
:100E430001C0804100C1814000C1814001C0804197
:100E530000C1814001C0804101C0804100C1814087
:100E630000C0C101C30302C2C60607C705C5C40447
:100E7300CC0C0DCD0FCFCE0E0ACACB0BC90908C8B7
:100E8300D81819D91BDBDA1A1EDEDF1FDD1D1CDCA7
:100E930014D4D515D71716D6D21213D311D1D01017
:100EA300F03031F133F3F23236F6F737F53534F407
:100EB3003CFCFD3DFF3F3EFEFA3A3BFB39F9F83877
:100EC30028E8E929EB2B2AEAEE2E2FEF2DEDEC2C67
:100ED300E42425E527E7E62622E2E323E12120E0D7
:100EE300A06061A163A3A26266A6A767A56564A4C7
:100EF3006CACAD6DAF6F6EAEAA6A6BAB69A9A86837
:100F030078B8B979BB7B7ABABE7E7FBF7DBDBC7C26
:100F1300B47475B577B7B67672B2B373B17170B096
:100F23005090915193535292965657975595945486
:100F33009C5C5D9D5F9F9E5E5A9A9B5B99595898F6
:100F4300884849894B8B8A4A4E8E8F4F8D4D4C8CE6
:100F53004484854587474686824243834181804056
:07238A0044024D00000000B9
:03000B000221646B
:10216400C0E0C0F0C083C082C0D075D000C000C041
:1021740004C005C006C007758CF8758ACD90024D61
:10218400E0FCA3E0FDA3E0FEA3E02401FFE43EFEA7
:10219400E43DFDE43CFC90024D12194DD007D006FD
:1021A400D005D004D000D0D0D082D083D0F0D0E0FD
:0121B40032F8
:030003000221FDDA
:1021FD00C0E0C0F0C083C082C0D075D000C000C0A8
:10220D0001C002C003C004C005C006C007D2001241
:10221D001BA7D007D006D005D004D003D002D00123
:0D222D00D000D0D0D082D083D0F0D0E032ED
:1023D400438901758CF8758ACDD28CD2B9D2A922E1
:05000600C288D2A8220F
:1023AF00C0A8C2AF90024DE0FCA3E0FDA3E0FEA3E6
:0423BF00E0FFD0A8C3
:0123C30022F7
:1014530090FFFC12195912194DC0A8C2AF85088319
:10146300850982E0FCA3E0FDA3E0FEA3E0FFFBAA65
:1014730006A905A80490024DE0FCA3E0FDA3E0FE4D
:10148300A3E0C39BFBEE9AFAED99F9EC98F8900070
:101493000412197DE0FEA3E0FFE4FCFDC312193C36
:1014A3004003021536850883850982E0FCA3E0FD2D
:1014B300A3E0FEA3E0FBAA06A905A80490024DE061
:1014C300FCA3E0FDA3E0FEA3E0C39BFFEE9AFEEDC9
:1014D30099FDEC98FCE4FBFAF9F8D312193C405857
:1014E300850883850982E0FCA3E0FDA3E0FEA3E079
:1014F300FBAA06A905A80490024DE0FCA3E0FDA306
:10150300E0FEA3E09BFFEE9AFEED99FDEC98FCEF65
:1015130024FFFBEE34FFFAED34FFF9EC34FFF890CF
:10152300000412197DE0FEA3E0FFE4FCFDC31219E1
:101533003C4005D0A8D38003D0A8C3C0D0900006F8
:06154300121959D0D0225C
:101FE50090FFFD121959EBF0A3EAF0A3E9F090FF79
:041FF500FD12195967
:101FF90090000312197DE0F9A3E0FAA3E0850883B4
:10200900850982C9F0A3EAF0A3E9F0850883850967
:1020190082E0FBA3E0FAA3E0F91218C36010850877
:1020290083850982A3E475F00112191080DD9000FF
:102039000312197DA3A3E0FF850883850982A3A361
:04204900E0C39FFF52
:06204D0090000602195983
:10236100EF1FAA0670011E4A6013E4FCFDC3ED9441
:0D23710051EC940450EA0DBD00010C80F009
:01237E00223C
:1017F90090FFFE121959EAF0A3EBF090FFFE1219BF
:1018090059ECF0A3EDF090FFFE121959EEF0A3EF99
:07181900F090FFFA121959CB
:1018200090000612197DE0FFA3E0850883850982F8
:10183000A3A3CFF0A3EFF090000812197DE0FEA360
:10184000E0FF90000412197DEEF0A3EFF090000A83
:1018500012197DE0FEA3E0FF850883850982A3A31A
:10186000E0FCA3E02FFFEC3E850883850982F0A30E
:10187000EFF0850883850982A3A3E0FEA3E0FF853E
:101880000883850982E0FCA3E06F7002EC6E602D96
:1018900090000412197DE475F00112192685F0827A
:1018A000F583E493FF850883850982A3A3E475F09B
:0D18B0000112192685F082F583EFF080B556
:0618BD0090000C02195915
:05172B00E0FEA3E0FF59
:1017300090FFFE121959EAF0A3EBF090FFFE121988
:1017400059ECF0A3EDF090FFFE121959EEF0A3EF63
:07175000F090FFFA12195995
:1017570090000612197DE0FFA3E0850883850982C2
:10176700A3A3CFF0A3EFF090000812197DE0FEA32A
:10177700E0FF90000412197DEEF0A3EFF090000A4D
:1017870012197DE0FEA3E0FF850883850982A3A3E4
:10179700E0FCA3E02FFFEC3E850883850982F0A3D8
:1017A700EFF0850883850982A3A3E0FEA3E0FF8508
:1017B7000883850982E0FCA3E06F7002EC6E602C61
:1017C70090000412197DE475F00112192685F08244
:1017D700F583E0FF850883850982A3A3E475F001FB
:0C17E70012192685F082F583EFF080B621
:0617F30090000C021959E0
:101E320090FFFF121959EDF090FFFE121959EEF0C2
:091E4200A3EFF090FFFE12195904
:101E4B00850883850982A3A3E0FEA3E0AA06F97B9C
:101E5B00FF121FE5850883850982E4F0A3EFF08567
:101E6B000883850982E0FEA3E0D39428EE9400401A
:101E7B000C850883850982E4F0A37428F085088318
:101E8B00850982E0FAA3E0FB850883850982A3A379
:101E9B00E0FCA3E0FD7E027F251217F990000412EF
:101EAB00197DE06019850883850982E0FAA3E0FBC0
:0E1EBB007C027D257E007F09120F631223C476
:061EC9009000050219590A
:101D940090FFFE121959EEF0A3EFF090FFFE121916
:011DA40059E5
:101DA500C0A8C2AF850883850982A3A3E0FEA3E08E
:101DB500FF2404F582E43EF583E0FCA3E0FDFBEFA0
:101DC5002406F582E43EF583E0FEA3E0C39BFFEE27
:101DD5009C850883850982F0A3EFF0850883850932
:101DE50082A3A3E0FEA3E0FF2406F582E43EF5838B
:101DF500E0FAA3E0FBD3ED9BEC9A401ED0A88F82BE
:101E05008E83A3A3E0FEA3E02401FFE43E850883BF
:101E15008509828FF01219108002D0A88508838564
:071E25000982E0FEA3E0FFCB
:061E2C00900004021959A8
:1022740090FFFE121959EEF0A3EFF085088385094B
:1022840082E0FEA3E0FF121D94850883850982E0A5
:10229400FCA3E0F5828C83A3A3E0FCA3E0C39FFF2F
:0922A400EC9EFE900002021959A3
:100F630090FFFE121959EAF0A3EBF090FFFE12195D
:100F730059ECF0A3EDF090FFFE121959EEF0A3EF38
:070F8300F090FFFC12195968
:100F8A0090000412197DE0FEA3E0FF122274850886
:100F9A0083850982EEF0A3EFF090000812197DE034
:100FAA00FEA3E0FF850883850982E0FCA3E0FDC378
:100FBA009FEC9E500B90000812197DECF0A3EDF007
:100FCA0090000412197DE0FEA3E0FFF5828E83A350
:100FDA00A3E0FCA3E0FD8F828E83E0FEA3E02DFF59
:100FEA00EE3CCF2401CF3400FE90000412197DE0BC
:100FFA00FCA3E02406F582E43CF583E0FCA3E0FDD3
:10100A00C3EF9DFFEE9C850883850982A3A3F0A305
:10101A00EFF090000812197DE0FEA3E0FF85088337
:10102A00850982A3A3E0FAA3E0FBC39FEA9E505C72
:10103A0090000612197DE0FCA3E0FD90000412194D
:10104A007DE0FEA3E02406F582E43EF58312172B29
:10105A00850883850982A3A3E0FEA3E0FF90000828
:10106A0012197DE0FCA3E0C39FFBEC9EFA900006F8
:10107A0012197DE0FCA3E02FFDEC3EFC9000041267
:10108A00197DE0FEA3E0F5828E8380289000081285
:10109A00197DE0FAA3E0FB90000612197DE0FCA39B
:1010AA00E0FD90000412197DE0FEA3E02406F5821B
:1010BA00E43EF58312172BC0A8C2AF90000812199C
:1010CA007DE0FEA3E0FF90000412197DE0FCA3E09E
:1010DA00FD2406F582E43CF583EE8FF01219108D9B
:1010EA00828C83A3A3E0FEA3E0FF8D828C83E0FCC5
:1010FA00A3E02FFDEC3ECD2401CD3400FC9000048A
:10110A0012197DE0FAA3E02406F582E43AF583E0B9
:10111A00FAA3E0C39DEA9C402890000412197DE0DE
:10112A00FCA3E0FDEF2401FFE43EFEC3E49FFFE4DD
:10113A009EFEED2406F582E43CF583EE8FF012194B
:0E114A0010D0A890000812197DE0FEA3E0FF6F
:0611580090000A02195983
:100B400090FFFE121959EAF0A3EBF090FFFE121984
:100B500059ECF0A3EDF090FFFE121959EEF0A3EF5F
:070B6000F090FFFC1219598F
:100B670090000412197DE0FEA3E0FF121D94850892
:100B770083850982EEF0A3EFF090000812197DE05B
:100B8700FEA3E0FF850883850982E0FCA3E0FDC39F
:100B97009FEC9E500B90000812197DECF0A3EDF02E
:100BA70090000412197DE0FEA3E0FFF5828E83A377
:100BB700A3E0FCA3E0FD8F828E83E0FEA3E02DFF80
:100BC700EE3CCF2401CF3400FE90000412197DE0E3
:100BD700FCA3E02404F582E43CF583E0FCA3E0FDFC
:100BE700C3EF9DFFEE9C850883850982A3A3F0A32D
:100BF700EFF090000812197DE0FEA3E0FF8508835F
:100C0700850982A3A3E0FAA3E0FBC39FEA9E507382
:100C170090000412197DE0FEA3E02404F582E43E6F
:100C2700F583E0FCA3E0FD90000612197D12172B57
:100C3700850883850982A3A3E0FEA3E0FF9000084F
:100C470012197DE0FCA3E0C39FFBEC9EFA90000421
:100C570012197DE0FEA3E0F5828E83E0FCA3E0FDA0
:100C6700850883850982A3A3E0FEA3E0FF90000621
:100C770012197DE0F8A3E0F58288832FFFE5833E14
:100C8700FE802D90000812197DE0FAA3E0FB90008A
:100C97000412197DE0FEA3E02404F582E43EF58307
:100CA700E0FCA3E0FD90000612197DE0FEA3E0FF43
:100CB70012173090000A12197DE06003020D52C02E
:100CC700A8C2AF90000812197DE0FEA3E0FF9000D4
:100CD7000412197DE0FCA3E0FD2404F582E43CF551
:100CE70083EE8FF01219108D828C83A3A3E0FEA3ED
:100CF700E0FF8D828C83E0FCA3E02FFDEC3ECD244A
:100D070001CD3400FC90000412197DE0FAA3E02421
:100D170004F582E43AF583E0FAA3E0C39DEA9C4038
:100D27002890000412197DE0FCA3E0FDEF2401FFE9
:100D3700E43EFEC3E49FFFE49EFEED2404F582E457
:100D47003CF583EE8FF0121910D0A8900008121905
:060D57007DE0FEA3E0FFB9
:060D5D0090000B02195981
:101AF90090FFFE121959EAF0A3EBF090FFFE1219BC
:101B090059ECF0A3EDF090FFFE121959EEF0A3EF96
:071B1900F090FFFD121959C5
:101B200090000712197DE0FCA3E0FDEC8508838599
:101B30000982F0A3EDF090000512197D74FFF5F015
:101B400012192645F0604D90000312197DE475F0DE
:101B50000112192685F082F583E0FF850883850947
:101B600082E06FA3A3F0850883850982A3A3E0FF29
:101B7000900D6393FE850883850982A3E06E850836
:101B800083850982F0EF900E63938508838509822F
:101B9000A3F080A2850883850982E0FEA3E0FDED25
:011BA000FF45
:061BA10090000902195931
:081ECF00900290EEF0A3EFF089
:101ED700E4FFAE038EC3900294E0602C75C7817552
:101EE700C501AE051DEE606DAE070F8EC475C65AEF
:101EF70075C6A500900290E475F00112192685F0C9
:101F070082F583E5C2F080DA8FC475C78175C50392
:101F170075C65A75C6A500E4F5C6F5C5F5C775C7F4
:101F27008175C5027C00ED1DAA0470011C4A60255D
:101F3700AE070F8EC4900290E475F0011219268542
:101F4700F082F583E0F5C275C65A75C6A500EF7035
:101F5700D505C380D1E4F5C6F5C5F5C775C3FF75CB
:021F6700C4FFB5
:011F69002255
:06239100C1004101D10072
:0E23F3007580007594FFE4900190F0A3F02235
:07240C0043A204759DFF22AD
:1022E300EF5407FFE4F5BCF5BDF5BEEF44E8F5BCDC
:1022F30000000000000000000000E5BC30E4FBE546
:10230300BD5403FEADBE7C00E42DFFEC3EFE53BC8A
:01231300EFDA
:0123140022A6
:02231500A90716
:10231700E4FFEFC39D501DEBA807088002C313D845
:10232700FC5401FEE92F24D3F582E43401F583EE52
:07233700F00F80DE02223AE4
:10223A00E4FFFEFDEF25E0FFEE33FEEDFBC374176E
:10224A009BFBE49400FA74D32BF58274013AF5836C
:10225A00E02FFFE43EFE0DEDB408D9EEF4900190B4
:09226A00F0A3EFF580F4FFF00091
:012273002248
:10233E007F189001D3E4F0A3DFFC9001EE7401F05E
:10234E00A37401F0A374E3F07F10900215E4F0A3E0
:02235E00DFFCA2
:01236000225A
:10088E00E490027AF0A37408F090027BE0FFD39418
:10089E0000402390027AE025E0F074D22FF582E436
:1008AE003401F583E0600790027AE04401F0900293
:1008BE007BE014F080D3E5A0F4900279F0A3E0FF82
:1008CE00900279E06F7003020B3F7F0A7E001223C5
:1008DE0061E5A0F4FD900279E0AF056D6003020BB7
:1008EE003FA3E06F5D1582F0E490027BF090027BF7
:1008FE00E0FFC39408501CED5401FE74D32FF58213
:10090E00E43401F583EEF0EDC313FD90027BE004B9
:10091E00F080DA9001A7E0F470289001A6E00000C4
:10092E00000000000000900279E030E00BE490013E
:10093E00A7F09001A6E004F0900279E0FFC313F057
:10094E008015900279E0FF5401FE9001A7E02EF091
:10095E00EFC313900279F09001A9E0F47028900192
:10096E00A8E00000000000000000900279E030E0F6
:10097E000BE49001A9F09001A8E004F0900279E058
:10098E00FFC313F08015900279E0FF5401FE900131
:10099E00A9E02EF0EFC313900279F09001ABE0F4D2
:1009AE0070289001AAE000000000000000009002F4
:1009BE0079E030E00BE49001ABF09001AAE004F096
:1009CE00900279E0FFC313F08015900279E0FF5496
:1009DE0001FE9001ABE02EF0EFC313900279F09080
:1009EE0001ADE0F470289001ACE0000000000000C2
:1009FE000000900279E030E00BE49001ADF0900140
:100A0E00ACE004F0900279E0FFC313F08015900281
:100A1E0079E0FF5401FE9001ADE02EF0EFC313908C
:100A2E000279F09001AFE0F470289001AEE0000082
:100A3E00000000000000900279E030E00BE490012D
:100A4E00AFF09001AEE004F0900279E0FFC313F036
:100A5E008015900279E0FF5401FE9001AFE02EF078
:100A6E00EFC313900279F09001B1E0F47028900179
:100A7E00B0E00000000000000000900279E030E0DD
:100A8E000BE49001B1F09001B0E004F0900279E037
:100A9E00FFC313F08015900279E0FF5401FE900120
:100AAE00B1E02EF0EFC313900279F09001B3E0F4B1
:100ABE0070289001B2E000000000000000009002DB
:100ACE0079E030E00BE49001B3F09001B2E004F075
:100ADE00900279E0FFC313F08015900279E0FF5485
:100AEE0001FE9001B3E02EF0EFC313900279F09067
:100AFE0001B5E0F470269001B4E0000000000000A3
:100B0E000000900279E030E00BE49001B5F0900126
:100B1E00B4E004F0900279E0C313F022900279E081
:100B2E00FF5401FE9001B5E02EF0EFC31390027951
:010B3E00F0C6
:010B3F002293
:10198A0012199F12199F12199F12199F12199F1249
:05199A00199F12199FC6
:10199F009001EDE0F9700EFF1222E3AA06EA54035C
:1019AF009002158070E9B4010F7F011222E3AA069D
:1019BF00EA5403900217805DE9B4020F7F021222EE
:1019CF00E3AA06EA5403900219804AE9B4030F7F91
:1019DF00031222E3AA06EA540390021B8037E9B4EC
:1019EF00040F7F041222E3AA06EA540390021D801B
:1019FF0024E9B4050F7F051222E3AA06EA540390E7
:101A0F00021F8011E9B406187F061222E3AA06EA24
:101A1F005403900221F0A3EFF09001EDE004F022C7
:101A2F00E9B407167F071222E3AA06EA54039002CD
:0A1A3F0023F0A3EFF0E49001EDF0B6
:011A4900227A
:101C4F0090015EE064016003021CF390FFFE121925
:101C5F0059E4F0A3740AF0900167E0FCA3E0FDA340
:101C6F00E0FEA3E0FF121453507AE490015EF07E81
:101C7F00007F01121D94D3EF9400EE940040659005
:101C8F00FFFF121959E4F0FA7B247C017DF17E00ED
:101C9F007F01120B40900279EFF07AFF7BFF24FE59
:101CAF00FDE434FFFC7E017FF1121AF9900279E016
:101CBF0024EFF582E43401F583E0FCA3E0B50724BB
:101CCF00ECB5062090019CE0FF9001F1E0FEB50716
:101CDF0002800BEEB4FF0D9001F2E0B40306900109
:041CEF00D27401F0BA
:011CF30022CE
:1022AD009001F2E04480F0A37401F07AFF7BFF7C93
:1022BD00007D037E017FF1121AF9AC06EC9001F45A
:1022CD00F0A3EFF07A007B057C017DF17E007F09A4
:0622DD00120F630223C48E
:05002600900279EFF0EB
:10002B00900288600D7401F0A37401F0A374ECF0DE
:10003B00800B7401F0A37401F0A374D2F0900288CA
:10004B00E0FBA3E0FAA3E0F91218C3700302088DDA
:10005B009001F2E024FE6026147003022420147039
:10006B000302025A1470030203DE14700302077EAC
:10007B0024F77003020567240E600302087B9001CE
:10008B00F3E0FF90027AE4F0A3EFF0E07F00FE9044
:10009B00027AF0A3EFF09001F4E0FDEDFF90027A0D
:1000AB00EEF0A3EFF0E004F0700690027AE004F0BB
:1000BB009001F5E0FF90027CE4F0A3EFF0E07F000D
:1000CB00FE90027CF0A3EFF09001F6E0FDEDFF90C7
:202420009001F4E0B47003022508B4750302243302066D90019CE09001F1F0A37403F074EA
:2024400008A3F0907FF9E493B4FF0B907FFFE493B4FF03022498907FF9E4939001F4F09027
:202460007FFAE4939001F5F0907FFBE4939001F6F0907FFCE4939001F7F0907FFDE49390F1
:2024800001F8F0907FFEE4939001F9F0907FFFE4939001FAF00224D790BFF9E4939001F414
:2024A000F090BFFAE4939001F5F090BFFBE4939001F6F090BFFCE4939001F7F090BFFDE454
:2024C000939001F8F090BFFEE4939001F9F090BFFFE4939001FAF0E4A3F07AFF7BFF7C008C
:2024E0007D0B7E017FF1121AF990027EEEF0A3EFF090027EE0FCA3E0FDEC9001FCF0A3ED6B
:20250000F07A007B0D02086990019CE09001F1F0A37403F07404A3F07406A3F07400A3F0AE
:202520007404A3F07400A3F07AFF7BFF7C007D077E017FF1121AF990027EEEF0A3EFF09082
:16254000027EE0FCA3E0FDEC9001F8F0A3EDF07A007B0902086953
:1000DB00027CEEF0A3EFF090027AE0FEA3E0FFC308
:1000EB009401EE9400500302087BA3E0FCA3E0FD17
:1000FB00EF2DFFEE3CFED3EF9419EE94004003027C
:10010B00087B90019CE09001F1F090027DE024FFD0
:10011B00FF90027CE034FFFEEF7803CEC313CE13C7
:10012B00D8F92401FFE43E900284F0A3EFF0900194
:10013B00F3F0E4900286F0A3F0FBFAD3900285E093
:10014B009B900284E09A5003020207E4900282F033
:10015B00900280F0A3F0900280E0FEA3E0FFC39436
:10016B0008EE9400506F900286E0FCA3E0FDEF2DAB
:10017B00FFEE3CFED390027DE09F90027CE09E4020
:10018B005490027AA3E0FF900287E02FFF90028643
:10019B00E03400FE900280E0FCA3E0FD2FFFEC3E7C
:1001AB00FE74D22FF58274013EF583E06017900246
:1001BB0082E0FFAE057401A806088002C333D8FCA9
:1001CB004F900282F0900281E004F07089900280DF
:1001DB00E004F08081900282E0FF74F42BF58274CE
:1001EB00013AF583EFF0900287E02408F090028645
:1001FB00E03400F00BBB00010A0201467AFF7BFFE3
:10020B00900285E02403FD900284E03400FC7E0123
:10021B007FF1121AF990027EEEF0A3EFF090027EBE
:10022B00E0FCA3E0FDECFF900284E0FAA3E0FB24EA
:10023B00F4F58274013AF583EFF074F52BF58274C3
:10024B00013AF583EDF0EB2405FBE43A02077790D6
:10025B0001F3E0FF90027AE4F0A3EFF0E07F00FE01
:10026B0090027AF0A3EFF09001F4E0FDEDFF900225
:10027B007AEEF0A3EFF0E004F0700690027AE0045F
:10028B00F09001F5E0FF90027CE4F0A3EFF0E07F4B
:10029B0000FE90027CF0A3EFF09001F6E0FDEDFF85
:1002AB0090027CEEF0A3EFF090027AE0FEA3E0FF69
:1002BB00C39401EE940050030203DBEF9409EE9418
:1002CB000040030203DBA3E0FEA3E0FF9408EE94DF
:1002DB000040030203DB90019CE09001F1F0A3745A
:1002EB0004F0EF25E0A3F0E4900280F0A3F090027D
:1002FB007CE0FEA3E0FFC3900281E09F900280E0D0
:10030B009E5074E0FEA3E0FF90027BE02FFF900273
:10031B007AE03EFEEF25E0FDEE33FC74132DF58203
:10032B0074023CF583E0FB900281E025E0FF900234
:10033B0080E033FE74F42FF58274013EF583EBF00D
:10034B0074132DF58274023CF583A3E0FD900281BA
:10035B00E025E0FF900280E033FE74F52FF5827408
:10036B00013EF583EDF0900281E004F070069002FF
:10037B0080E004F00202F97AFF7BFF9001F3E024A6
:10038B0003FDE433FC7E017FF1121AF990027EEE3D
:10039B00F0A3EFF090027EE0FD900281E025E0FFFC
:1003AB00900280E033FE74F42FF58274013EF583E6
:1003BB00EDF090027EA3E0FD74F52FF58274013E03
:1003CB00F583EDF09001F3E02405FBE433020777AE
:1003DB0002087B9001F3E0FF90027AE4F0A3EFF0C8
:1003EB00E07F00FE90027AF0A3EFF09001F4E0FDC5
:1003FB00EDFF90027AEEF0A3EFF0E004F0700690C0
:10040B00027AE004F090027AE0FEA3E0FFC39411BD
:10041B00EE94005003020564EF9419EE9400400330
:10042B000205649001F5E0FDF4706990027AA3E097
:10043B0024EF900282F09001EEE0FBA3E0FAA3E040
:10044B00F9900282E0FFF58275830074011218EEB9
:10045B00EF7005D280020503EFB40105D2810205CE
:10046B0003EFB40205D282020503EFB40305D28376
:10047B00020503EFB40404D284807DEFB40504D2EB
:10048B00858075EFB40604D286806DEF64077068C3
:10049B00D2878064ED706190027AA3E024EF900222
:1004AB0082F09001EEE0FBA3E0FAA3E0F990028268
:1004BB00E0FFF582758300E41218EEEF7004C28042
:1004CB008036EFB40104C281802EEFB40204C282E5
:1004DB008026EFB40304C283801EEFB40404C284ED
:1004EB008016EFB40504C285800EEFB40604C286F5
:1004FB008006EFB40702C28790019CE09001F1F0F7
:10050B00A37405F07AFF7BFF7C007D067E017FF1F3
:10051B00121AF990027EEEF0A3EFF090027EE0FC4F
:10052B00A3E0FDEC9001F7F0A3EDF07A007B087CE3
:10053B00017DF17E007F09120F631223C4900279B3
:10054B00E0700302087E900282E02493F582E4348B
:10055B0001F5837401F002087E02087B9001F3E041
:10056B00FF90027AE4F0A3EFF0E07F00FE90027AB6
:10057B00F0A3EFF09001F4E0FDEDFF90027AEEF0C6
:10058B00A3EFF09001F5E0FF90027CE4F0A3EFF015
:10059B00E07F00FE90027CF0A3EFF09001F6E0FD0F
:1005AB00EDFF90027CEEF0A3EFF090027AE0FEA359
:1005BB00E0FFC39410EE9400500302066AA3E0FC24
:1005CB00A3E0FDEF2DFFEE3CFED3EF9418EE94006D
:1005DB00400302066A9001F7E0B4010E90027AA381
:1005EB00E0FF9001F8E0FB12231590019CE09001D5
:1005FB00F1F0A3740FF07AFF7BFF7C007D067E0188
:10060B007FF1121AF990027EEEF0A3EFF090027ECA
:10061B00E0FCA3E0FDEC9001F7F0A3EDF07A007B9A
:10062B00087C017DF17E007F09120F631223C490B9
:10063B000279E0700302087E900283E0FF90027C57
:10064B00A3E0FEC3EF9EFEEEC39F400302087E7441
:10065B00822EF582E43401F5837401F00E80E802FA
:10066B00087B9001F3E0FF90027AE4F0A3EFF0E057
:10067B007F00FE90027AF0A3EFF09001F4E0FDED25
:10068B00FF90027AEEF0A3EFF0E004F07006900218
:10069B007AE004F09001F5E0FF90027CE4F0A3EF28
:1006AB00F0E07F00FE90027CF0A3EFF09001F6E00B
:1006BB00FDEDFF90027CEEF0A3EFF090027AE0FEEE
:1006CB00A3E0FFC39440EE9400500302077BA3E02A
:1006DB00FCA3E0FDEF2DFFEE3CFED3EF944DEE942B
:1006EB0000400302077B90019CE09001F1F0A374A2
:1006FB0003F0ED25E0FFA3EFF0FB7A00C0029002C0
:10070B007BE025E0FF90027AE033FE741C2FF97436
:10071B00013EFCAD017E017FF4D0021217307AFF4F
:10072B007BFF9001F3E02403FDE433FC7E017FF1BA
:10073B00121AF990027EEEF0A3EFF090027EE0FC2D
:10074B00A3E0FDECFF9001F3E024F4F582E4340127
:10075B00F583EFF09001F3E024F5F582E43401F535
:10076B0083EDF09001F3E02405FBE433FA02086912
:10077B0002087B9001F3E0FF90027AE4F0A3EFF024
:10078B00E07F00FE90027AF0A3EFF09001F4E0FD21
:10079B00EDFF90027AEEF0A3EFF0E004F07006901C
:1007AB00027AE004F090027AE0FEA3E0FFC39440EB
:1007BB00EE94005003020879EF944DEE9400400341
:1007CB000208797C017DF5EF25E0FFEE33FE7437EF
:1007DB002FF974013EFEAF017A007B0212173090A5
:1007EB0001A0E09001BBF07E017FB6E4900294F093
:1007FB00FB7D1B121ECF7A007B1A7C017DB77E011D
:10080B007F9C12173090019CE09001F1F0A37406CD
:10081B00F090027BE025E0FF90027AE033FE743724
:10082B002FF974013EFCAD017E017FF57A007B024E
:10083B001217307AFF7BFF7C007D067E017FF11261
:10084B001AF990027EEEF0A3EFF090027EE0FCA38B
:10085B00E0FDEC9001F7F0A3EDF07A007B087C0152
:10086B007DF17E007F09120F631223C48005800087
:10087B001222AD900288E0FBA3E0FAA3E0F9E412A8
:02088B0018DC77
:01088D002248
:10154900E4FE74452EF582E43401F583E0FD74D39D
:101559002EF582E43401F583E0FC6D601974452EA3
:10156900F582E43401F583ECF074882EF582E434D5
:1015790001F5837401F00EEEB408C7E4FEEE25E030
:10158900244EF582E43401F583E0FCA3E0FDEE2569
:10159900E02415F582E43402F583E0FAA3E0FBD3F5
:1015A9009DEA9C401AEE25E0244EF582E43401F5CB
:1015B90083A3E0FDC3EB9DFFD39401406F803EEE12
:1015C90025E0244EF582E43401F583E0FCA3E0FD37
:1015D900EE25E02415F582E43402F583E0FAA3E070
:1015E900FBC39DEA9C5045EE25E0244EF582E43488
:1015F90001F583A3E0C39BFFD39401402FEE25E0BF
:101609002415F582E43402F583E0FCA3E0FDEE2520
:10161900E0244EF582E43401F583ECF0A3EDF07497
:101629006B2EF582E43401F5837401F00EEE640843
:051639006003021586AC
:01163E002289
:101BA7007E017FB69002947401F0E4FB7D1B121E48
:101BB700CF9001B6E0B4AB0A9001BBE0B41E03308E
:101BC70000769001B674ABF0A37401F0E4A3F0A320
:101BD700F0A37407F0A3741EF0E49001C0F0900125
:101BE700BFF09001BEF09001BDF09001D0F09001E0
:101BF700CFF09001CEF09001CDF09001CCF09001A4
:101C0700CBF09001CAF09001C9F09001C8F09001A3
:101C1700C7F09001C6F09001C5F09001C4F09001A3
:101C2700C3F09001C2F09001C1F07E017FB690022F
:101C370094F0FB7D1B121ECF7A007B1A7C017DB7C7
:081C47007E017F9C1217302280
:0220B300AA067B
:1020B50090019EE09001F1F0A37405F0EAA3F0A36E
:1020C500EFF074D32DF582E43401F583E0600890D8
:1020D50001F574FFF08005E49001F5F0E49001F658
:1020E500F07AFF7BFFFC7D067E017FF1121AF9ACC9
:1020F50006EC9001F7F0A3EFF07A007B087C017DF8
:0B210500F17E007F09120F631223C45B
:0121100022AC
:1021B500E4900279F0900279E0FFC39408503874F6
:1021C500882FF582E43401F583E06023900279E0FD
:1021D500FD2410FFE433FE1220B3900279E0248839
:1021E500F582E43401F583E4F07FC8FE12236190A3
:0721F5000279E004F080BE56
:0121FC0022C0
:10115E00E4900279F09001A2E0FF90027BE4F0A30C
:10116E00EFF0E07F00FE90027BF0A3EFF09001A382
:10117E00E0FDEDFF90027BEEF0A3EFF0E490027A3B
:10118E00F09001A4E0FF90027DE4F0A3EFF0E07F89
:10119E0000FE90027DF0A3EFF09001A5E0FDEDFFC3
:1011AE0090027DEEF0A3EFF090027BE0FEA3E0FF55
:1011BE004E605AA3E0FCA3E0FD4C6051D3EF9DEED0
:1011CE009C400890027BECF0A3EDF090027BE0FED9
:1011DE00A3E0FF4E700302128B90FFFE121959EE20
:1011EE00F0A3EFF090015FE0FCA3E0FDA3E0FEA30F
:1011FE00E0FF121453400302128B1223AF90015FD3
:10120E0012194D9002797401F0A3F0807090027B58
:10121E00E0FEA3E0FF4E602D90FFFE121959EEF096
:10122E00A3EFF090015FE0FCA3E0FDA3E0FEA3E0DE
:10123E00FF121453500F1223AF90015F12194D90ED
:10124E0002797401F090027DE0FEA3E0FF4E602D66
:10125E0090FFFE121959EEF0A3EFF0900163E0FC3F
:10126E00A3E0FDA3E0FEA3E0FF121453500F1223E0
:10127E00AF90016312194D90027A7401F0900279C9
:10128E00E0FF64016009A3E064016003021337907C
:10129E00019CE09001F1F0A37404F0EF640170166C
:1012AE0090027AE0B4010F9001F37410F07A00FB13
:1012BE007C027D15801B9001F37402F0900279E0A0
:1012CE007A007B02B401067C027D1580047C027DCF
:1012DE00177E017FF41217307AFF7BFF9001F3E047
:1012EE002403FDE433FC7E017FF1121AF9AD07AC45
:1012FE0006ECFF9001F3E024F4F582E43401F5836B
:10130E00EFF09001F3E024F5F582E43401F583ED7E
:10131E00F09001F3E02405FBE433FA7C017DF17ECD
:09132E00007F09120F631223C4B1
:011337002293
:101A4A0075C13F9001D1E014604F046003021AF897
:101A5A001223D41200061223F312240C12233E126C
:101A6A001BA7C2B390019FE02436F582E43401F546
:101A7A0083E0F58D12088E12198A7FC87E00122320
:101A8A006175C13F9001D17401F01223AF900163D7
:101A9A0012194D90015F02194D90019BE0FF6009F8
:101AAA0064026005EF6401704590FFFE121959E463
:101ABA00F0A37419F0900141E0FCA3E0FDA3E0FE5D
:101ACA00A3E0FF121453501E1223AF9001411219C2
:101ADA004D12088E12198A90019DE060091215496B
:0F1AEA001221B512115E121C4FE4FF12002622CA
:0124130022A6
:0F23E40090015E7401F01223AF90016702194D52
:101D1400022401E493A3F8E493A34003F68001F2C0
:101D240008DFF48029E493A3F85407240CC8C333D0
:101D3400C4540F4420C8834004F456800146F6DF9F
:101D4400E4800B010204081020408090237FE47E8D
:101D5400019360BCA3FF543F30E509541FFEE49394
:101D6400A360010ECF54C025E060A840B8E493A35B
:101D7400FAE493A3F8E493A3C8C582C8CAC583CA86
:101D8400F0A3C8C582C8CAC583CADFE9DEE780BE3E
:012397000045
:1018C300BB010689828A83E0225002E722BBFE0223
:0918D300E32289828A83E4932256
:1018DC00BB010689828A83F0225002F722BBFE01EB
:0218EC00F322E5
:1018EE00F8BB010DE58229F582E5833AF583E8F030
:1018FE00225006E92582C8F622BBFE05E92582C8DC
:02190E00F222C3
:10191000C5F0F8A3E028F0C5F0F8E5821582700262
:061920001583E038F022FF
:10192600A3F8E0C5F025F0F0E58215827002158374
:06193600E0C838F0E822D1
:10193C00EB9FF5F0EA9E42F0E99D42F0E89C45F001
:01194C002278
:0C194D00ECF0A3EDF0A3EEF0A3EFF0220D
:10195900E5092582F582E5083583F583B50804850F
:1019690082092210AF06858209F50822858209F5C8
:0419790008D2AF22BF
:0D197D00E5092582F582E5083583F5832212
:00000001FF
